:100000000C947C000C9497000C9497000C9497002F
:100010000C9497000C9497000C9497000C94970004
:100020000C9497000C9497000C9497000C949700F4
:100030000C9497000C9497000C9497000C949700E4
:100040000C9497000C9497000C9497000C949700D4
:100050000C9497000C9497000C9497000C949700C4
:100060000C9497000C9497000C9497000C949700B4
:100070000C9497000C9497000C942C020C9497000D
:100080000C9497000C9497000C949700ED01E101FB
:10009000D501C901BD01B101A50199018D01FE0183
:1000A000FE01FE01FE01FE01FE01FE01810175015E
:1000B00069015D0151014501FE01FE01FE01FE01E4
:1000C000FE01FE01FE01FE01FE01FE01FE01FE0138
:1000D000FE01FE01FE01FE01FE01FE01FE01FE0128
:1000E000FE01FE01FE01FE01FE01FE01810175011E
:1000F00069015D015101450111241FBECFEFD0E11F
:10010000DEBFCDBF11E0A0E0B1E0EAE4F6E002C05E
:1001100005900D92A438B107D9F713E0A4E8B1E037
:1001200001C01D92A638B107E1F70C94B8000C94F9
:10013000000010928601109285010895F89480E0E5
:1001400090E00E940B0380936F0010929B0010922E
:100150009D0086E080939D001092980087E0809338
:10016000990010929A0088E980939A0078940895F3
:10017000CFEFD0E1DEBFCDBF0E949E008091850110
:100180008F3FE1F786E891E00E949E020E9499006D
:10019000F5CF80939C0021E030E080919B0099276F
:1001A00046E0969587954A95E1F7817090708217A1
:1001B000930799F780919B00806480939B0008953A
:1001C0001F93CF93DF93EC0110E08881882381F0A7
:1001D000FE01E10FF11D80810E94C9001F5F81E0D7
:1001E00090E00197F1F7FE01E10FF11D8081EECF64
:1001F0008AE00E94C90081E090E00197F1F78DE06C
:100200000E94C900DF91CF911F91089588E00E945C
:10021000C90081E090E00197F1F780E20E94C900F7
:1002200081E090E00197F1F788E00E94C90008950D
:100230001F93CF93DF93EC0150E0FC01019000206D
:10024000E9F731974E2F481B8881883719F0883598
:1002500009F0D9C0152F423008F4D0C0212F332720
:10026000FE01E20FF31F81819927AA27BB27FC011A
:10027000F197E633F10508F0C1C0EA5BFF4FEE0FDE
:10028000FF1F0590F491E02D0994842F9927821B7C
:10029000930B880F991F880F991F08972FE030E064
:1002A000A7C0842F9927821B930B880F991F880F53
:1002B000991F08972EE030E09BC0842F9927821B5E
:1002C000930B880F991F880F991F08972DE030E036
:1002D0008FC0842F9927821B930B880F991F880F3B
:1002E000991F08972CE030E083C0842F9927821B48
:1002F000930B880F991F880F991F08972BE030E008
:1003000077C0842F9927821B930B880F991F880F22
:10031000991F08972AE030E06BC0842F9927821B31
:10032000930B880F991F880F991F089729E030E0D9
:100330005FC0842F9927821B930B880F991F880F0A
:10034000991F089728E030E053C0842F9927821B1B
:10035000930B880F991F880F991F089727E030E0AB
:1003600047C0842F9927821B930B880F991F880FF2
:10037000991F089726E030E03BC0842F9927821B05
:10038000930B880F991F880F991F089725E030E07D
:100390002FC0842F9927821B930B880F991F880FDA
:1003A000991F089724E030E023C0842F9927821BEF
:1003B000930B880F991F880F991F089723E030E04F
:1003C00017C0842F9927821B930B880F991F880FC2
:1003D000991F089722E030E00BC0842F9927821BD9
:1003E000930B880F991F880F991F089721E030E021
:1003F00002C0220F331F8A95E2F7520F1F5F12309F
:1004000008F429CF23C0823611F08234D9F454176E
:10041000E8F4242F332761E070E021503040FE01E2
:10042000142F8191813341F4CB01022E02C0880F39
:10043000991F0A94E2F7582B115021503040112394
:1004400081F704C0CE010E94DE02582F852F992724
:10045000DF91CF911F9108951F920F920FB60F92C7
:1004600011242F933F934F935F936F937F938F93B9
:100470009F93AF93BF93EF93FF93809185018F3F3D
:1004800009F441C0E0918401AE2FBB27AA57BE4FAB
:1004900080919C008C938C91883041F40E940601DD
:1004A000809184018823C9F181502AC08C918A30BF
:1004B00029F08C918D3011F0EF3FB1F4EE23A1F0D3
:1004C000FF27EA57FE4F10828FEF8093850110922D
:1004D00084018AE00E94C90081E090E00197F1F771
:1004E0008DE00E94C90019C080918401E82FFF2788
:1004F000EA57FE4F80810E94C900809184018F5F7E
:10050000809384010AC080919C008A3031F08D3044
:1005100021F080E091E00E94E000FF91EF91BF9117
:10052000AF919F918F917F916F915F914F913F918B
:100530002F910F900FBE0F901F901895EF92FF9282
:100540000F931F938C0162E171E00E941B03892BC2
:1005500019F48AE291E009C06CE171E0C8010E94DF
:100560001B03892B29F486E491E00E94E0001FC060
:1005700082E691E00E94E00080E791E00E94E000C6
:10058000EE24FF248701F701EE0DFF1DEA5DFE4F0B
:10059000808191810E94E0000894E11CF11C011D02
:1005A000111D82E0E816F1040105110560F30E94B7
:1005B00099001F910F91FF90EF900895FC018827FB
:1005C0009927E89421912223F1F02032D9F32930A0
:1005D000C9F32A30B9F32C30A9F32D3099F326371B
:1005E00089F32B3219F02D3221F4689421912223C2
:1005F00051F0203344F02A3334F420530E94130383
:10060000820F911DF3CF8115910521F01EF4809585
:10061000909501960895E199FECF9FBB8EBBE09A1D
:1006200099278DB308957AE0979F902D879F802D0D
:10063000910D11240895FB01DC018D910190801929
:0A06400011F40020D1F7990B089582
:10064A0043657265626F74204E6F742052656164EF
:10065A007900436F6D6D616E64203100436F6D6D7B
:10066A00616E6420320012011C01436F6D6D616E70
:10067A0064203120686173206265656E2065786543
:10068A00637574656400436F6D6D616E642032201A
:10069A00686173206265656E206578656375746547
:1006AA006400436F6D6D616E64204572726F7200F3
:1006BA0056616C696420636F6D6D616E647320614D
:0406CA0072653A001B
:00000001FF
